:020000040000FA
:0400000024EF21F0D8
:08000800056ED8CF06F0E0CF31
:1000100007F00001E9CF0DF0EACF08F0E1CF09F0D9
:10002000E2CF0AF0D9CF0BF0DACF0CF0F3CF14F017
:10003000F4CF15F0FACF16F000C00FF001C010F0A9
:1000400002C011F003C012F004C013F0F2AA2CEFAA
:1000500000F0F2B4C2EF04F00FC000F010C001F0E5
:1000600011C002F012C003F013C004F00E8E0DC0D8
:10007000E9FF08C0EAFF09C0E1FF0AC0E2FF0BC0C8
:10008000D9FF0CC0DAFF14C0F3FF15C0F4FF16C08F
:10009000FAFF055007C0E0FF06C0D8FF1000F2CFFE
:1000A0000EF0F29EF76AB80FF66E000EF722090006
:1000B000F5500EBEF28E12000D0A82728263834AE0
:1000C000815B836882F08F898AFA89BB82B582C49A
:1000D00082A282DC82B982F120536920636F6D6D48
:1000E000616E6400F2CF0EF0F29EF76AFE0FF66EBC
:1000F000000EF7220900F5500EBEF28E12000D0A16
:1001000082728263834A815B836882CC826582606B
:1001100082738FEE95F182F093C782F182C582A23D
:1001200082DC82B982F18140536D20636F6D6D6115
:100130006E640000F2CF0EF0F29EF76A4E0FF66E7C
:10014000010EF7220900F5500EBEF28E12000D0AC4
:10015000838A815B83688272826382C5838A8367B4
:100160008389834382AA82A082E882DC82B582BD31
:1001700020256400F2CF0EF0F29EF76A8E0FF66E25
:10018000010EF7220900F5500EBEF28E12000D0A84
:100190006E6F2061636B20434D4432340000F2CF18
:1001A0000EF0F29EF76AB80FF66E010EF722090004
:1001B000F5500EBEF28E12005049433138462041B0
:1001C00044206C6F676765720000F2CF0EF0F29EFC
:1001D000F76AE40FF66E010EF7220900F5500EBE25
:1001E000F28E120046415433322053442043617250
:1001F000642020200000F2CF0EF0F29EF76A100F6C
:10020000F66E020EF7220900F5500EBEF28E1200B5
:1002100025356C64206D5620202020200000F2CF70
:100220000EF0F29EF76A380FF66E020EF722090002
:10023000F5500EBEF28E120025386C58207365639F
:10024000742025325800F2CF0EF0F29EF76A600F4C
:10025000F66E020EF7220900F5500EBEF28E120065
:100260000D0A504943313846323535302053442049
:1002700063617264206D6F6E69746F722032303109
:10028000322E342E37206275663D3078256C58004A
:10029000F2CF0EF0F29EF76AAA0FF66E020EF72268
:1002A0000900F5500EBEF28E12000D0A504943317E
:1002B00038465F4D4F4E3E00F2CF0EF0F29EF76A89
:1002C000D20FF66E020EF7220900F5500EBEF28E26
:1002D00012000D0A434D443920726573203D2025DC
:1002E00058200000F2CF0EF0F29EF76AFE0FF66E75
:1002F000020EF7220900F5500EBEF28E12000D0A12
:10030000434D44353520726573203D20255820002B
:10031000F2CF0EF0F29EF76A2A0FF66E030EF72266
:100320000900F5500EBEF28E12000D0A41434D44F5
:10033000313320726573203D202558200D0A0000BE
:10034000F2CF0EF0F29EF76A5A0FF66E030EF72206
:100350000900F5500EBEF28E12006C6F6720656EBC
:100360006400F2CF0EF0F29EF76A7C0FF66E030E79
:10037000F7220900F5500EBEF28E12000D0A6164DC
:100380006C6F67736571203D2025642C2061647259
:1003900065616470203D20256C580000F2CF0EF09E
:1003A000F29EF76AB60FF66E030EF7220900F550BB
:1003B0000EBEF28E12000D0A43757272656E7420C5
:1003C000736563746F72203D20256C580000F2CF76
:1003D0000EF0F29EF76AE80FF66E030EF7220900A0
:1003E000F5500EBEF28E12000D0A82658260827395
:1003F0008FEE95F182F093C782F182C582A282DCF2
:1004000082B982F10000F2CF0EF0F29EF76A200F5F
:10041000F66E040EF7220900F5500EBEF28E1200A1
:100420000D0A5344206973206E6F742072656164F5
:100430007900F2CF0EF0F29EF76A4C0FF66E040EC2
:10044000F7220900F5500EBEF28E12000D0A434D40
:1004500044303A200000F2CF0EF0F29EF76A700F9F
:10046000F66E040EF7220900F5500EBEF28E120051
:100470000D0A434D44383A200000F2CF0EF0F29EB0
:10048000F76A940FF66E040EF7220900F5500EBEBF
:10049000F28E12000D0A434D4435383A2000F2CF57
:1004A0000EF0F29EF76AB80FF66E040EF7220900FE
:1004B000F5500EBEF28E12000D0A41434D44343108
:1004C0003A200000F2CF0EF0F29EF76ADE0FF66ED1
:1004D000040EF7220900F5500EBEF28E12000D0A2E
:1004E000837483408343838B8341838D8350815BFB
:1004F0008356838783938386836A8362836782AA12
:1005000020307834302833326B422982C582CD8244
:10051000A082E882DC82B982F100F2CF0EF0F29E76
:10052000F76A340FF66E050EF7220900F5500EBE7D
:10053000F28E12000D0A46415433322082C582CD1C
:1005400082A082E882DC82B982F10000F2CF0EF054
:10055000F29EF76A660FF66E050EF7220900F55057
:100560000EBEF28E12000D0A8E7792E88CC2909425
:1005700082CC837483408343838B82F08DEC90AC78
:1005800082C582AB82DC82B982F1206D61783D3018
:1005900078256C580000F2CF0EF0F29EF76AB00F8B
:1005A000F66E050EF7220900F5500EBEF28E12000F
:1005B0000D0A82728263834A815B836882C9826585
:1005C000826082738252825182C5835F837E815BA7
:1005D000837483408343838B82F08DEC90AC82B52F
:1005E00082DC82B70D0A0000F2CF0EF0F29EF76AAD
:1005F000020FF66E060EF7220900F5500EBEF28EBF
:10060000120082B782D782C482CC83748340834332
:10061000838B82AA8DED8F9C82B382EA82DC82B7C3
:10062000814282E682EB82B582A282C582B782A92C
:10063000814820792F6E0000F2CF0EF0F29EF76A0B
:10064000520FF66E060EF7220900F5500EBEF28E1E
:1006500012000D0A726574203D2025580000F2CF6B
:100660000EF0F29EF76A780FF66E060EF72209007A
:10067000F5500EBEF28E12000D0A6E6F2061636B94
:1006800020434D4432350000F2CF0EF0F29EF76A5F
:10069000A20FF66E060EF7220900F5500EBEF28E7E
:1006A00012000D0A777269746520646174612830E4
:1006B0007846432C2E2E2E2920726573706F6E7330
:1006C00065206973206E6F742030785835206F7202
:1006D0002072656164790000F2CF0EF0F29EF76A35
:1006E000F20FF66E060EF7220900F5500EBEF28EDE
:1006F00012000D0A5344206572726F7220617420DB
:10070000736563743D256C582C7265743D255800E3
:10071000F2CF0EF0F29EF76A2A0FF66E070EF7225E
:100720000900F5500EBEF28E12000D0A7772697440
:1007300065206572726F722E20726573706F6E73B2
:1007400065203D20253032580000F2CF0EF0F29E99
:10075000F76A640FF66E070EF7220900F5500EBE19
:10076000F28E12000D0A4D42525F73746172742052
:100770003D203078256C582C204D42525F766F6CAE
:100780007365637473203D203078256C580D0A0022
:10079000F2CF0EF0F29EF76AAA0FF66E070EF7225E
:1007A0000900F5500EBEF28E12004D4252207061CB
:1007B000727469746F6E2074797065203D20307892
:1007C00025580D0A0000F2CF0EF0F29EF76AE00FF6
:1007D000F66E070EF7220900F5500EBEF28E1200DB
:1007E000464154305F7374617274203D2030782527
:1007F0006C582C204641545F73697A65203D203047
:1008000078256C5820736563746F72730D0A00004D
:10081000F2CF0EF0F29EF76A2A0FF66E080EF7225C
:100820000900F5500EBEF28E12004449525F7374F7
:1008300061727420203D203078256C582C2053653F
:1008400063746F72732070657220636C7573746566
:1008500072203D203078256C580D0A00F2CF0EF042
:10086000F29EF76A760FF66E080EF7220900F55031
:100870000EBEF28E120066696C652073746172742C
:10088000203D203078256C582C200000F2CF0EF04F
:10089000F29EF76AA60FF66E080EF7220900F550D1
:1008A0000EBEF28E120046415420747970652020ED
:1008B000203D2025730D0A00F2CF0EF0F29EF76A5C
:1008C000D20FF66E080EF7220900F5500EBEF28E1A
:1008D000120053442072656164206572726F722049
:1008E00020200000F2CF0EF0F29EF76AFE0FF66EA7
:1008F000080EF7220900F5500EBEF28E1200444990
:100900005220656E747279202000F2CF0EF0F29EB4
:10091000F76A240FF66E090EF7220900F5500EBE95
:10092000F28E12000D0A64617465203D20256C581A
:100930000000F2CF0EF0F29EF76A4C0FF66E090E31
:10094000F7220900F5500EBEF28E12004425303415
:100950006C752020205458542000F2CF0EF0F29EE7
:10096000F76A740FF66E090EF7220900F5500EBEF5
:10097000F28E12000D0A636F6D6D616E64206572F8
:10098000726F7200D76A830ED66E0601ED2BF9875F
:10099000F12BD8B4F22BED51040806E2ED6BEE2BEF
:1009A000EF2BD8B4F02BF981FDA134D0FDA332D0C8
:1009B000C282C2B2FED7C4CFBBF70701C3CFBAF71A
:1009C0000601FFC603F0FE51FE2BD8B4FF2B070132
:1009D000BC6F230EBC25E96E000E0320EA6EBAC779
:1009E000EFFF0601FE530BE1FF51040808E1FD5142
:1009F000100B01E1FD87040EFF6F0C0EFE6FFF511F
:100A0000050808E2020EFF6F0C0EFE6FFD51080B89
:100A100001E1FD89EE510908D8B064D0ED53D8A4A6
:100A200061D0EE6BF983F72BF751090853E2F98592
:100A3000F76BF82B212A21503B084CE2216A202A2F
:100A400020503B0847E2206A1F2A1F50170842E245
:100A50001F6A1E2A1D50020A000109E0060A20E052
:100A6000020A1EE00F0A1CE0020A1AE022D01B5004
:100A7000030B0701BC6FBD6BBC530AE1BD5308E11A
:100A80001E501D0804E2010E1E6E030E1D6E07D0DF
:100A90001E501C0804E2010E1E6E030E1D6E19D0BE
:100AA0001E501E0803E2010E1E6E1D2A070111D002
:100AB00000011E501F080BE2010E1E6E1D2A1D5064
:100AC0000C0805E2010E1D6E1B2AD8B41C2A070172
:100AD00000D0060108C709F707C708F706C707F7D8
:100AE00082CF06F7F29400012CEF00F00701AEBFB1
:100AF00010D00F0E006EAD3900160A0E005C03E236
:100B0000300E002602D0AE51002600509EA8FED71F
:100B1000AD6E0F0EAD170A0EAD5D02E2300E02D0C3
:100B2000AE9FAE51AD27AD519EA8FED7AD6E000170
:100B3000000C070EEA6E6C0EE96EEF500EE0050E2B
:100B4000016E006A002EFED7012EFBD72E0E006E1E
:100B5000002EFED700D0EF2EF2D7000C080E016E4B
:100B6000040E006E002EFED78A969396040E006E39
:100B7000002EFED70701A5378A980DE39388040E4F
:100B8000006E002EFED781B807D0020E016E93864C
:100B9000938829D001D093980000938681A6FED730
:100BA000012E01D002D00001DBD7040E006E002E12
:100BB000FED78A96939600009388040E006E002E4E
:100BC000FED7040E006E002EFED7938681A6FED7B8
:100BD000016A040E006E002EFED781B801808A964D
:100BE00093968A98939800000001000C9388040E55
:100BF000006E002EFED79386040E006E002EFED7E8
:100C0000060E006E81A6FCD781A8FAD7002EFAD76F
:100C10008A989398040E006E002EFED78A969396BB
:100C2000000E186E7C0E0701A56F000197DF07010B
:100C3000A56B000193DFA1C7A5F790DF9398000093
:100C4000938681A6FED7040E006E002EFED700D03C
:100C500000009388040E006E002EFED7000C2A0EB2
:100C600007016A6F280E6C6F000163DF380E070101
:100C7000A16F0001BBDF390E0701A16F0001B6DFD4
:100C8000140E0701A16F0001B1DF07016A510F0BBC
:100C900070096B6FA16F0001A9DF07016A39006E4F
:100CA0000F0E00160050030B5C096C6FA16F000162
:100CB0009DDF6C0E0701A16F000198DF020E070196
:100CC0006B6F960E6C6F000134DF07016B2FF9D745
:100CD000380EA16F00018ADF0C0E0701A16F000121
:100CE00085DF010E0701A16F000180DF020E070101
:100CF0006C6F00011EDF000E016E000C9388040E65
:100D0000006E002EFED79386040E006E002EFED7D6
:100D1000060E006E81A6FCD781A8FAD7002EFAD75E
:100D20008A989398040E006E002EFED78A969396AA
:100D3000000E186E7C0E0701A56F00010FDF400E3C
:100D40000701A56F00010ADFA4C7A5F707DF939885
:100D50000000938681A6FED7040E006E002EFED7FB
:100D600000D000009388040E006E002EFED7D1EF55
:100D700006F0A2C703F00701A1C7E9FFA2C7EAFF77
:100D8000EF5211E0A2C703F0A151A12BD8B4A22BBE
:100D9000E96E03C0EAFFEFCFA3F7A3C7A4F70001F2
:100DA000ADD7E7D707010001000C800E0701A16F46
:100DB00000011CDF07016A6B6A510F0816E3170E6A
:100DC0006A25036A2F0FE96E070E0320EA6E036A95
:100DD0006A51F2CF70F7F29E0001CFEC00F00701EC
:100DE00070BFF28EEF6E6A2BE7D7566B070E6C6FF3
:100DF000460E6B6F6CC7A2F76BC7A1F70001B9DF96
:100E0000C00E0701A16F0001F1DE07016A6B6A5194
:100E10000F0816E3170E6A25036A2F0FE96E070EF7
:100E20000320EA6E036A6A51F2CF70F7F29E000166
:100E3000E5EC00F0070170BFF28EEF6E6A2BE7D78A
:100E4000070E6C6F460E6B6F6CC7A2F76BC7A1F7EE
:100E500000018FDF000E016E000C0701A06B9F6B7D
:100E6000BC0E1B5CA16F070E1C58000E9F59000E94
:100E7000A059D890996B9A6B9B6BA1359C6F9E6B18
:100E8000006A016A1D34026E9E35036E0236033617
:100E9000023603360236033602360336E00E0216F9
:100EA0000050991301509A1302509B1303509C1346
:100EB0009E6B006A016A0050991301509A131E50EC
:100EC0009B139E519C139F6B9E6B006A1F34016E97
:100ED0009E35026E9F35036E0136023603360136AB
:100EE00002360336F80E01160050991301509A137A
:100EF00002509B1303509C13A06B9F6B9E6B20347E
:100F0000006E9E35016E9F35026EA035036E003671
:100F10000136023603360036013602360336003615
:100F20000136023603360036013602360336E00E4D
:100F300000160050991301509A1302509B1303504E
:100F40009C13A06B9F6B9E6BD890A031036E9F315A
:100F5000026E9E31016E2130991301509A13025096
:100F60009B1303509C1399C700F09AC701F09BC7CD
:100F700002F09CC703F00001000C0701AD6BAE6BE3
:100F8000010EAF6FDA6AD96A070EB26FA50EB16FA4
:100F9000070EEA6EA90EE96EB2C7E2FFB1C7E1FF24
:100FA000AFC7B0F7D890E550EE02F350AD23F45040
:100FB000AE23B02FF7D7ADC7DEFFAEC7ADF7AE6B30
:100FC000D8B0AE2BB12BD8B4B22BAF2BAF51050894
:100FD000DFE10001000C006A016A026A036A07018E
:100FE000B56BB66BB76BB86BB451B311B211B1112D
:100FF0002CE0200EB96FD890AD37AE37AF37B03791
:10100000B537B637B737B837B451B85D08E1B35123
:10101000B75D05E1B251B65D02E1B151B55D0FE3D7
:10102000B151B55FB251D8A0B23DB65FB351D8A0AF
:10103000B33DB75FB451D8A0B43DB85FD880003697
:10104000013602360336B92FD6D7070EEA6EB50E33
:10105000E96E0001000C58C7EAFF57C7E9FF070116
:10106000ADC7EFFFE92AD8B4EA2AEF6A572BD8B404
:10107000582B0001000CE9500701A56FA4AF0DD05B
:10108000A507A58BA11FA21FA31FA41FA12BD8B426
:10109000A22BD8B4A32BD8B4A42B3B0EAC6F9A0EC2
:1010A000AB6FCA0EAA6FA96B0A0EA76FA4C7B0F7E1
:1010B000A3C7AFF7A2C7AEF7A1C7ADF7ACC7B4F7E8
:1010C000ABC7B3F7AAC7B2F7A9C7B1F7000183DF6F
:1010D0000150EFCFA1F7ECCFA2F7ECCFA3F7ECCF05
:1010E000A4F7005213E10701A751010AD8A402D0C6
:1010F00000010CD0A5510DE00F0BA75D01E02BE224
:10110000A5BF29D0A5BD05D0200E1FD0200E0701F8
:10111000A517A5AB0BD0A59B00C0A5F72D0EAD6FF5
:10112000000199DF0701A5C700F0A56B300EA5AB44
:101130000CD0A59B00C0A5F72D0EAD6F00018BDF75
:101140000701A5C700F0A56B300E002600C0ADF763
:10115000000181DF0701ACC7B0F7ABC7AFF7AAC783
:10116000AEF7A9C7ADF7B46BB36BB26B0A0EB16F34
:10117000000131DF03C0ACF702C0ABF701C0AAF732
:1011800000C0A9F70701A72F91D7000109EF09F0C7
:101190000701A46BA36B9CC7A2F79BC7A1F7A4C7C9
:1011A000A8F7A3C7A7F79CC7A6F79BC7A5F7AC6B83
:1011B000AB6B130EAA6FEC0EA96F0001DEDE03C04D
:1011C000A0F702C09FF701C09EF700C09DF707017E
:1011D0009EC79DF79FC79EF7A0C79FF7A06BA03340
:1011E0009F339E339D33A0339F339E339D333F0EF9
:1011F000A017070E586F460E576F050EE96EA0C771
:10120000A4F79FC7A3F79EC7A2F79DC7A1F7000148
:1012100032D7040E0701A16FA1510001FBEC00F0D1
:101220000701A12B006EAD6F000115DF0C0E070149
:10123000A15DF2E1C00EA16F0001D8DC070E07012D
:10124000A26F460EA16F000194DD000E016E000C2E
:101250000701B05302E0938401D093940001000C85
:101260000701B66B9392B76BB751070813E3D89099
:10127000B637B5AF02D0948001D09490938281A00C
:1012800001D0B62BD890B537B751070801E093923B
:10129000B72BEAD7B6C701F00001000C0701B06B0D
:1012A0000001D6DFABC7B5F7DBDFAFC7B1F707018A
:1012B000B26BB36BB46BAFC7B5F70001D1DFAEC78C
:1012C000B1F7AFC7B2F70701B36BB46BAEC7B5F7F1
:1012D0000001C6DFADC7B1F7AEC7B2F7AFC7B3F70E
:1012E0000701B46BADC7B5F70001BADFACC7B5F7FE
:1012F000B7DF950E0701B56F0001B2DFFF0E0701E2
:10130000B56F0001ADDF0150000C010E0701A26FA7
:101310009B2D48D199C701F09AC703F099C7A3F74D
:101320009AC7A4F799C7E9FF9AC7EAFFEFCFA7F7D3
:10133000ECCFA8F7ECCFA9F7ECCFAAF7510EAB6F23
:10134000AAC7AFF7A9C7AEF7A8C7ADF7A7C7ACF74D
:101350000001A4DF07019D6B9C6B9D5318E19C511C
:10136000630815E3FF0EB56F00017ADF07019F6B7D
:1013700001C09EF79E51800BA36FA46BA35303E1A2
:10138000A45301E104D09C2BD8B49D2BE6D79D6BD0
:101390009C6B9D5103081DE303E19C51E70819E391
:1013A000FF0EB56F00015CDF07019F6B01C09EF768
:1013B0009E3D02D09F5301E00CD09EAA06D09EAA6B
:1013C000FED7AE50030801E104D09C2BD8B49D2B6E
:1013D000E0D79E51FE0803E19F53D8B472D0A253C8
:1013E00008E0A207A2517D0803E30601FC2B0701D8
:1013F00091D7010EB06F00012BDFFF0E0701B56F13
:1014000000012EDF070199C701F09AC703F099C7C1
:10141000A3F79AC7A4F799C7E9FF9AC7EAFFEFCFE6
:10142000A7F7ECCFA8F7ECCFA9F7ECCFAAF7AB6BF7
:10143000AB5100016CEC03F00701AB2B006E0050C8
:101440009EA8FED7AD6E130EAB5DF2E1AAC7ADF755
:10145000370EAE6F000176EC05F0A9C7ADF7370E79
:101460000701AE6F000176EC05F0A8C7ADF7370EA7
:101470000701AE6F000176EC05F0A7C7ADF7370E98
:101480000701AE6F000176EC05F0160E0701AC6F98
:10149000AC5100016CEC03F00701AC2B006E005066
:1014A0009EA8FED7AD6E1B0EAC5DF2E19EC7ADF7F8
:1014B000370EAE6F000176EC05F0FF0E016EA9D27B
:1014C00007010C0E9925016E000E9A21036E01C0D2
:1014D000A3F7A46F01C0E9FFEA6EEF2C2FD0A16B38
:1014E000A06BA151010829E3040E9925016E000E9D
:1014F0009A21036E01C0A3F7A46F01C0E9FFEA6E51
:10150000ECCFA8F7ED52EFCFA7F7A751A025016EBA
:10151000A851A121036E01C0A9F7AA6FFF0EB56FF4
:1015200000019EDEAAC7EAFFA9C7E9FF01C0EFFFDD
:101530000701A02BD8B4A12BD4D71DD0A16BA06BD1
:10154000A151010818E3230EA025016E000EA12170
:10155000036E01C0A3F7A46FFF0EB56F000180DE1C
:10156000A4C7EAFFA3C7E9FF01C0EFFF0701A02B53
:10157000D8B4A12BE5D7FF0EB56F000171DEFF0EC9
:101580000701B56F00016CDE010E0701B06F0001AD
:101590005FDEFF0E0701B56F000162DE000E016E17
:1015A00038D207019B510208D8A4FCD099C701F09A
:1015B0009AC703F099C7A3F79AC7A4F799C7E9FF99
:1015C0009AC7EAFFEFCFA7F7ECCFA8F7ECCFA9F7C0
:1015D000ECCFAAF7580EAB6FAAC7AFF7A9C7AEF703
:1015E000A8C7ADF7A7C7ACF7000158DE07019D6B90
:1015F0009C6B9D5314E19C51630811E3FF0EB56F82
:1016000000012EDE07019F6B01C09EF79E5303E190
:101610009F5301E104D09C2BD8B49D2BEAD7FE0E3A
:10162000B56F00011DDE0C0E07019925016E000E3D
:101630009A21036E01C0A3F7A46F01C0E9FFEA6E0F
:10164000EF2C28D0A16BA06BA151010822E3040E5E
:101650009925016E000E9A21036E01C0A3F7A46FB5
:1016600001C0E9FFEA6EECCFA8F7ED52EFCFA7F784
:10167000A751A025E96EA851A121EA6EEFCFA9F7E5
:10168000A9C7B5F70001ECDD0701A02BD8B4A12B49
:10169000DBD716D0A16BA06BA151010811E3230E7B
:1016A000A025E96E000EA121EA6EEFCFA3F7A3C734
:1016B000B5F70001D5DD0701A02BD8B4A12BECD7DD
:1016C000010EB56F0001CCDD010E0701B56F000101
:1016D000C7DD07019D6B9C6BFF0EB56F0001C0DD80
:1016E00007019F6B01C09EF79E3D02D09F5305E00E
:1016F0009FC79DF79EC79CF709D09EAA06D09EAAB9
:10170000FED7AE50030801E101D0E6D7FF0EB56F5A
:101710000001A6DD07019F6B01C09EF79E3D03D02F
:101720009F5301E109D09EAA06D09EAAFED7AE50D3
:10173000030801E101D0EAD79C51E50802E19D537D
:1017400017E0A36BA351000188EC03F00701A32B62
:10175000006E00509EA8FED7AD6E1A0EA35DF2E19A
:101760009CC7ADF7370EAE6F000176EC05F00701B0
:10177000010EB06F00016CDDFF0E0701B56F0001B7
:101780006FDD07019C51E50808E19D5306E1010E5C
:10179000016E00013ED105D00701000E016E00016F
:1017A00038D107019B51050844E199C701F09AC758
:1017B00003F099C7A3F79AC7A4F799C7E9FF9AC797
:1017C000EAFFEFCFA7F7ECCFA8F7ECCFA9F7ECCF64
:1017D000AAF7590EAB6FAAC7AFF7A9C7AEF7A8C74C
:1017E000ADF7A7C7ACF7000159DD07019D6B9C6BF6
:1017F000FF0EB56F000134DD07019F6B01C09EF73E
:101800009E5303E19F5301E10FD09EAA09D09EAAE7
:10181000FED7AE50030804E19F6BFF0E9E6F04D00D
:101820009C2BD8B49D2BE4D79EC701F00001F1D0CA
:1018300007019B510608D8A4AED0B06B000108DDAB
:10184000FC0E0701B56F00010BDD0C0E0701992599
:10185000016E000E9A21036E01C0A3F7A46F01C0B0
:10186000E9FFEA6EEF2C28D0A16BA06BA151010813
:1018700022E3040E9925016E000E9A21036E01C029
:10188000A3F7A46F01C0E9FFEA6EECCFA8F7ED5211
:10189000EFCFA7F7A751A025E96EA851A121EA6EC5
:1018A000EFCFA9F7A9C7B5F70001DADC0701A02B34
:1018B000D8B4A12BDBD716D0A16BA06BA151010826
:1018C00011E3230EA025E96E000EA121EA6EEFCFF1
:1018D000A3F7A3C7B5F70001C3DC0701A02BD8B459
:1018E000A12BECD79D6B9C6BFF0EB56F0001B8DC94
:1018F00007019F6B01C09EF79E511F0BA36FA46B46
:10190000A351050803E1A45301E10FD09EAA09D019
:101910009EAAFED7AE50030804E19F6BFF0E9E6F98
:1019200004D09C2BD8B49D2BDFD79E3D07D09F536E
:1019300005E19EC701F000016CD007019D6B9C6B17
:10194000FF0EB56F00018CDC07019F6B01C09EF795
:101950009E3D03D09F5301E10FD09EAA09D09EAABD
:10196000FED7AE50030804E19F6B030E9E6F04D0B8
:101970009C2BD8B49D2BE4D79E3D08D09F5306E105
:10198000010E016E000145D005D00701030E016E66
:1019900000013FD007019B5107083CE1FD0EB56FE8
:1019A00000015EDC07019D6B9C6BFF0EB56F0001B3
:1019B00057DC07019F6B01C09EF79E3D03D09F53EC
:1019C00001E10FD09EAA09D09EAAFED7AE5003080F
:1019D00004E19F6B030E9E6F04D09C2BD8B49D2B0B
:1019E000E4D7010EB06F000133DCFF0E0701B56FC5
:1019F000000136DC07019E3D08D09F5306E1010E31
:101A0000016E000106D005D00701030E016E000132
:101A100000D007010001000C0701A0BF12D00F0E7B
:101A2000006E9F3900160A0E005C03E2300E00269D
:101A300002D0A051002600C0ADF700012BEC08F049
:101A400007010F0E9F170A0E9F5D02E2300E02D0B3
:101A5000A09FA0519F279FC7ADF700012BEC08F076
:101A6000000C070E0701586F460E576F9CC79FF773
:101A7000370EA06F0001D0DF9BC79FF7370E07011D
:101A8000A06F0001C9DF9AC79FF7370E0701A06F4B
:101A90000001C2DF99C79FF7370E0701A06F000151
:101AA000BBDF040E07019E6F9E5100010FEC01F099
:101AB00007019E2B006EAD6F00012BEC08F00A0EA3
:101AC00007019E5DF1E19DC79FF7370EA06F0001F2
:101AD000A3DF800E0701A16F0001F6EC05F0070EF1
:101AE0000701A26F460EA16F0001B9EC06F0000ECF
:101AF000016E000C9EAA05D09EAAFED7AECF01F0C3
:101B000094D10601F9A18FD1F991FDA155D1FDA381
:101B100053D107010451010A000104E0020AD8B4BC
:101B200045D149D10601FD51180BD8B43DD103C7A9
:101B300022F702C721F701C720F700C71FF7FDA74B
:101B400073D0020E07019A6F230E9AC798F7976F0A
:101B500000012DEC07F003C096F702C095F701C015
:101B600094F700C093F70C0E07019725E96E000E5D
:101B70009821EA6EEFCF00F0ECCF01F0ECCF02F04D
:101B8000ECCF03F001C09AF700C099F701C09CF7B1
:101B900000C09BF70001C8EC08F0070198C703F0EC
:101BA00097C700F0040E9727D8B0982B00C0E9FF24
:101BB00003C0EAFF93C7EFFF94C7ECFF95C7ECFFA4
:101BC00096C7ECFF98C703F097C700F0040E97275D
:101BD000D8B0982B00C0E9FF03C0EAFF00C7EFFFB1
:101BE00001C7ECFF02C7ECFF03C7ECFF98C703F087
:101BF00097C700F0040E9727D8B0982B00C0E9FFD4
:101C000003C0EAFF0601F351F55D006EF451F65989
:101C100000C0EFFFEC6EEC6AEC6A020E0701246F65
:101C2000230E236F74D00601FDA971D0040E0701A5
:101C30009A6F230E9AC798F7976F00012DEC07F063
:101C400003C096F702C095F701C094F700C093F760
:101C50000C0E07019725E96E000E9821EA6EEFCF72
:101C600000F0ECCF01F0ECCF02F0ECCF03F001C0BC
:101C70009AF700C099F701C09CF700C09BF70001DC
:101C8000C8EC08F0070198C703F097C700F0040EEE
:101C90009727D8B0982B00C0E9FF03C0EAFF93C78D
:101CA000EFFF94C7ECFF95C7ECFF96C7ECFF98C712
:101CB00003F097C700F0040E9727D8B0982B00C008
:101CC000E9FF03C0EAFF00C7EFFF01C7ECFF02C74F
:101CD000ECFF03C7ECFF98C703F097C700F0040EB2
:101CE0009727D8B0982B00C0E9FF03C0EAFF060190
:101CF000F351F55D006EF451F65900C0EFFFEC6E44
:101D0000EC6AEC6A040E0701246F230E236F010EA8
:101D100007012B6FF2C6F4F6F1C6F3F6070E9A6FC1
:101D20001F0E996F020E9B6F000185EC09F001C038
:101D300090F7F2C6F6F6F1C6F5F60701905311E1F9
:101D4000996B99510001BAEC00F00701992B006ED4
:101D500000509EA8FED7AD6E0E0E995DF2E1046BA9
:101D600003D0030E046F056BE70E0601FD17FB534E
:101D70000AE0010E07010027D8B0012BD8B4022BCE
:101D8000D8B4032B06D0020E07010127000E022350
:101D9000032303C79CF702C79BF701C79AF700C745
:101DA00099F79D6B00015DDE000105D0010E070172
:101DB000046F000100D00601070107510615926F5C
:101DC00009510811916F92A30AD09151020B07E1BA
:101DD000010E0A6F1B0E016E000127D0070192A5AC
:101DE0000AD09151040B07E1020E0A6F1B0E016E1F
:101DF00000011BD0070192A90AD09151100B07E1F5
:101E0000040E0A6F1B0E016E00010FD0070192AB8A
:101E10000AD09151200B07E1050E0A6F1B0E016ECF
:101E2000000103D00701000165D620EF0FF0070184
:101E30008C6B8D6B8C518A5DD8A079D000015AD6FD
:101E400001C08EF707018E51030803E1FF0E016EFA
:101E500078D08E511B080BE10A5309E088C7E9FFCF
:101E600089C7EAFF1B0EEF6E010E016E6AD08E511C
:101E70000D080BE1036A8D518825E96E8951032015
:101E8000EA6EEF6A8DC701F05CD08E51080803E05E
:101E90008E517F081BE18C5319E08D518C5D16E14A
:101EA0008C518C07036A8825E96E89510320EA6EFC
:101EB000EF6A8D07080E9EA8FED7AD6E200E9EA875
:101EC000FED7AD6E080E9EA8FED7AD6E8B2D06D048
:101ED0008E51720803E1720E016E33D08B2D06D045
:101EE0008E516E0803E16E0E016E2BD08E517F0B6A
:101EF0001F081CE28E517F0B7E0818E38D518C5D0C
:101F000015E18C518C2B036A8825E96E89510320D9
:101F1000EA6E8EC7EFFF8EC78FF78F519EA8FED750
:101F2000AD6E8C518D5D02E28CC78DF783D7036A4D
:101F30008C518825E96E89510320EA6EEF6A8DC7BE
:101F400001F00001000C070180518009836FA16F2F
:101F50000001F6EC05F082C7A2F781C7A1F7B9EC42
:101F600006F0000E016E000CE9500701846F3B0E75
:101F70008B6F9A0E8A6FCA0E896F886B0A0E866FF6
:101F800083C7B0F782C7AFF781C7AEF780C7ADF799
:101F90008BC7B4F78AC7B3F789C7B2F788C7B1F759
:101FA0000001EBEC07F00150EFCF80F7ECCF81F7A9
:101FB000ECCF82F7ECCF83F7005213E10701865193
:101FC000010AD8A402D000010CD084510CE00F0B00
:101FD000865D01E00EE284BF0CD084BD04D0200EEB
:101FE00003D00701846B300E002600509EA8FED758
:101FF000AD6E8BC7B0F78AC7AFF789C7AEF788C792
:10200000ADF7B46BB36BB26B0A0EB16F0001EBECC2
:1020100007F003C08BF702C08AF701C089F700C040
:1020200088F70701862FACD7000138EF11F00601C1
:10203000895306E18A5304E18B5302E18C5305E096
:10204000200E07017E6F04D00601A1C67EF70701AE
:102050006C5303E06DC773F701D0736B7E51735DF2
:10206000D8B081D2A0C612F79FC611F79EC610F74E
:102070009DC60FF773510F27000E10231123122353
:102080000601FB530CE1D89011C712F710C711F7E6
:102090000FC710F707010F6B103711371237070101
:1020A000146B230E136F186B010E176F1B6F070E47
:1020B0009A6F0F0E996F010E9B6F000185EC09F06E
:1020C00001C06FF707016F51FF0839E1070E586F24
:1020D000460E576F806B805100015CEC04F00701E5
:1020E000802B006EAD6F00012BEC08F0100E070185
:1020F000805DF1E16C5318E1070EEA6E460EE96E61
:10210000000EEF1008E0EF509EA8FED7AD6EE92A52
:10211000D8B4EA2AF5D70D0E9EA8FED7AD6E0A0EEA
:102120009EA8FED7AD6E08D0806B070E826F460E5C
:10213000816F000108DF0701FF0E016E16D26C539C
:1021400003E06EC76FF701D06F6B6F510F08D8A017
:1021500008D2756B6FC774F7743775377437753776
:10216000743775377437753774377537E00E7417F1
:10217000230E7425E96E000E7521EA6EEFCF70F71D
:102180000B0E7425806F000E7521816F230E802544
:10219000E96E000E8121EA6EEFCF71F771511008E0
:1021A00003E1010E7F6F01D07F6B70512F0803E2B6
:1021B0007051390808E270514008D8B0C1D170514F
:1021C0005A08D8A0BDD17151200804E071511008FF
:1021D000D8A4B6D10D0E9EA8FED7AD6E0A0E9EA84D
:1021E000FED7AD6E796B786B776B766B1C0E7425B2
:1021F000806F000E7521816F230E8025016E000E09
:10220000812101C07AF77B6F7AC7E9FF7BC7EAFFBC
:10221000EFCF00F0ECCF01F0ECCF02F0ECCF03F009
:1022200003C079F702C078F701C077F700C076F7EE
:102230006C5323E17F5310E0806B8051000172ECFE
:1022400004F00701802B006E00509EA8FED7AD6EF3
:102250000B0E805DF2E111D04A0EE96E79C783F76B
:1022600078C782F777C781F776C780F700017CD6F9
:10227000200E9EA8FED7AD6E0701140E7425806F48
:10228000000E7521816F230E8025016E000E8121C5
:1022900001C07CF77D6F7CC7E9FF7DC7EAFFECCF0B
:1022A00003F0ED52EFCF00F003C001F0026A036AC1
:1022B00003C079F702C078F701C077F700C076F75E
:1022C00077C779F776C778F7766B776B060E7C253C
:1022D000E96E000E7D21EA6EECCF03F0ED52EF5077
:1022E000762703507723000E782379230601C15106
:1022F0000701765F0601C2510701775B0601C351F2
:102300000701785B0601C4510701795B79C7A8F71B
:1023100078C7A7F777C7A6F776C7A5F7A4C6ACF71F
:10232000A3C6ABF7A2C6AAF7A1C6A9F70001BDECE8
:1023300007F003C079F702C078F701C077F700C053
:1023400076F70601895306E18A5304E18B5302E1D3
:102350008C5311E0B951070176270601BA510701E4
:1023600077230601BB51070178230601BC51070101
:10237000792310D006019D510701762706019E5151
:102380000701772306019F51070178230601A05119
:10239000070179236C5324E179C7ADF7370EAE6F8F
:1023A000000176EC05F078C7ADF7370E0701AE6F88
:1023B000000176EC05F077C7ADF7370E0701AE6F79
:1023C000000176EC05F076C7ADF7370E0701AE6F6A
:1023D000000176EC05F0200E9EA8FED7AD6E070139
:1023E000716B7151070846E371517425806F000EBF
:1023F0007521816F230E8025E96E000E8121EA6E22
:10240000EFCF72F77251200803E16C5301E132D033
:102410006C5313E171517425806F000E7521816F2B
:10242000230E8025E96E000E8121EA6EEFCF82F740
:1024300082519EA8FED7AD6E1BD0170E7125036A80
:102440002F0F016E070E032271517425836F000E4A
:102450007521846F230E8325E96E000E8421EA6EB8
:10246000EFCF85F703C0EAFF01C0E9FF85C7EFFFA3
:10247000712BB7D7080E7427000E7523230E742511
:10248000E96E000E7521EA6EEF50200854E06C539F
:102490002FE12E0E9EA8FED7AD6E716B7151020812
:1024A00026E371517425806F000E7521816F230E14
:1024B0008025E96E000E8121EA6EEFCF72F772512E
:1024C000200801E114D071517425806F000E752130
:1024D000816F230E8025E96E000E8121EA6EEFCF19
:1024E00082F782519EA8FED7AD6E712BD7D723D02D
:1024F0002E0E4E6F716B715102081DE3200E712577
:10250000036A2F0F016E070E032271517425836F2A
:10251000000E7521846F230E8325E96E000E842141
:10252000EA6EEFCF85F703C0EAFF01C0E9FF85C778
:10253000EFFF712BE0D76C5303E0010E016E15D055
:102540009EAA0DD09EAAFED7AE50030802E10BD082
:1025500006D09EAAFED7AE50030801E104D06F2B2F
:10256000F4D5732B7BD5000E016E0001000C070122
:102570007351016A725D03E272C700F00CD0006A09
:10258000080E746F723700367351005CD8B0006E5D
:102590000136742FF7D70001000C200E07016DA93A
:1025A000300E6E6F6CC700F06CAF07D0001E002AB3
:1025B00000C06CF72D0E6E6F6D8F01506CC772F7F7
:1025C000640E736F0001D3DF00C06CF7300E01247E
:1025D00007016F6F6CC772F70A0E736F0001C7DFD8
:1025E000300E00240701716F300E0124706F6EC72A
:1025F00000F06DA702D06DAF6D956DB90BD06DAFCA
:1026000022D06DB520D000C06FF76DB31CD000C0D4
:1026100070F719D0300E6F5D16E100C06FF7200E15
:102620006E6F6DA704D06D956D836DAF6D93300E99
:10263000705D09E100C070F7200E6F6F6DA7F7D7CE
:102640006D936DAF6D916DA506D06EC7ADF70001AE
:102650002BEC08F007016DA306D06FC7ADF70001A2
:102660002BEC08F007016DA105D070C7ADF7000194
:102670002BEC08F071C7ADF700012BEC08F0000C53
:1026800007010B2D97D06A51010A000105E0030AEA
:1026900034E0010A67E08DD007010C6B0D6B0E6B07
:1026A000010E6C6F0CC76DF70DC76EF70001BFDC34
:1026B00001C06BF707016B2D1ED0070E586F520E2D
:1026C000576F200EAD6F00012BEC08F00EC76CF7B2
:1026D000110E07016D6F000160DF4D0E0701AD6F38
:1026E00000012BEC08F00701806B070E826F460E8D
:1026F000816F000128DC00015CD007010D2B0D511A
:102700000F0801E20D6B0E6B010E6C6F0CC76DF7BD
:102710000DC76EF700018BDC01C06BF707016B2D55
:102720001FD0070E586F520E576F200EAD6F00016D
:102730002BEC08F00EC76CF7110E07016D6F00014E
:102740002CDF4D0E0701AD6F00012BEC08F00701E7
:10275000806B070E826F460E816F0001A3EC0FF0B5
:10276000000127D0040E07010E270E511F0801E2B9
:102770000E6B070E586F520E576F200EAD6F000193
:102780002BEC08F00EC76CF7110E07016D6F0001FE
:1027900004DF4D0E0701AD6F00012BEC08F00701BF
:1027A000806B070E826F460E816F0001A3EC0FF065
:1027B00000D007010001000C0D0E9EA8FED7AD6EE3
:1027C0000A0E9EA8FED7AD6E000C070192512F088D
:1027D00007E29251390804E392510F0B016E10D0B9
:1027E00092AB02D04F0E92179251400807E29251DD
:1027F000460804E3370E925D016E02D0FF0E016EB3
:102800000001000C0701726B280E7B6F7B517B0768
:10281000000AD8B4B5D0766B756B746B736B7B5153
:102820007B07000AD8B492D06BC703F06A516A2BB9
:10283000D8B46B2BE96E03C0EAFFEFCF70F76F538C
:1028400034E170C792F70001C0DF01C071F70701E2
:10285000713D16D07251722B040DF350036A6C2532
:10286000016E6D51032201C0E9FF03C0EAFF73C787
:10287000EFFF74C7ECFF75C7ECFF76C7ECFF66D0BF
:1028800073377437753776377337743775377637EC
:1028900073377437753776377337743775377637DC
:1028A000F00E73177151731350D070C792F7000177
:1028B0008CDF01C071F70701713D01D003D0715168
:1028C000090816E27251722B040DF350036A6C254D
:1028D000016E6D51032201C0E9FF03C0EAFF73C717
:1028E000EFFF74C7ECFF75C7ECFF76C7ECFF2ED087
:1028F00076C77AF775C779F774C778F773C777F72C
:102900007737783779377A377737783779377A374B
:10291000FC0E7717735177277451782375517923FB
:1029200076517A23D8907737783779377A377AC7DC
:1029300076F779C775F778C774F777C773F771516A
:102940007327000E74237523762369D770512008EE
:1029500002E070530BE16E51725D04E372C701F047
:102960000FD003D0FF0E016E0BD009D070512C0890
:1029700006E070512E0803E0FF0E016E01D046D72D
:102980000001000CEACF74F7E9CF73F707016DAFD0
:1029900008D0738F73A9732B6C1F6D1F6C2BD8B469
:1029A0006D2B6D39F0096F6F6F27E20F706F320F6B
:1029B000726F6D510F0B702770277227E90F716FBF
:1029C000712771276C390F0B712772277137723796
:1029D000721F72376C510F0B72276F37070E6E6FB5
:1029E0000A0E71077227FDE370077127FDE36F0779
:1029F0007027FDE36E076F27FDE3070EEA6E6E0E8C
:102A0000E96E070E7315739DE906731507E173B937
:102A1000E92A73B903D0200E006E1CD0E926720E8D
:102A2000E95CD8B4738DEF50006E08E173BD06D039
:102A300073B914D073B702D0200E0BD073AF06D089
:102A40002D0E006EED50739D739F04D073877399A4
:102A5000300E002600509EA8FED7AD6EEE5073AD2E
:102A6000DED700013BEF15F0020EE96E6BC76DF784
:102A70006AC76CF787D7200E9EA8FED7AD6E000CF4
:102A8000200E07016DA9300E6E6F6CC700F06CAFA1
:102A900007D0001E002A00C06CF72D0E6E6F6D8FE0
:102AA00001506CC772F7640E736F000160DD00C0E7
:102AB0006CF7300E012407016F6F6CC772F70A0EB6
:102AC000736F000154DD300E00240701716F300E6A
:102AD0000124706F6EC700F06DA702D06DAF6D95C9
:102AE0006DB90BD06DAF22D06DB520D000C06FF79F
:102AF0006DB31CD000C070F719D0300E6F5D16E1B9
:102B000000C06FF7200E6E6F6DA704D06D956D83BA
:102B10006DAF6D93300E705D09E100C070F7200E4F
:102B20006F6F6DA7F7D76D936DAF6D916DA504D0E5
:102B30006E519EA8FED7AD6E6DA304D06F519EA8B6
:102B4000FED7AD6E6DA104D070519EA8FED7AD6EBC
:102B500071519EA8FED7AD6E0001000C6AC76CF7DC
:102B6000010E07016D6F00018BDF2F0E9EA8FED7AF
:102B7000AD6E000C6BC7ADF7370E0701AE6F0001ED
:102B800076EC05F0000C0701B06B000128EC09F0B1
:102B90006AC7B5F730EC09F06EC771F70701726BC1
:102BA000736B746B6EC7B5F7000130EC09F06DC73D
:102BB00071F76EC772F70701736B746B6DC7B5F76A
:102BC000000130EC09F06CC771F76DC772F76EC782
:102BD00073F70701746B6CC7B5F7000130EC09F0AF
:102BE0006BC7B5F730EC09F06FC7B5F730EC09F0FB
:102BF000FF0E0701B56F000130EC09F001504AEFFC
:102C000025F06FC7ADF7370E0701AE6F000176EC08
:102C100005F06EC7ADF7370E0701AE6F000176EC19
:102C200005F0DAEF26F007016A6B6A510001ADEC9E
:102C300004F007016A2B006E00509EA8FED7AD6E0F
:102C40000F0E6A5DF2E10001000C0601FC5317E073
:102C500007016B6B6B5100019AEC00F007016B2BC5
:102C6000006E00509EA8FED7AD6E230E6B5DF2E1A4
:102C7000FCC66CF71F0E6D6F000102DF060100013C
:102C8000000CF0C62AF6EFC629F66BC79AF76AC79A
:102C900099F7050E07019B6F000185EC09F001C053
:102CA0006DF7F0C62CF6EFC62BF607016D5312E058
:102CB000726B725100012FEC03F00701722B006E52
:102CC00000509EA8FED7AD6E0E0E725DF2E1FF0EB3
:102CD000016EE2D06C5310E0040E6A25016E000E06
:102CE0006B2101C0E9FFEA6EECCF03F0ED52EFCFAC
:102CF0006EF703C06FF705D0736B230E73C76FF7C2
:102D00006E6F080E6A25016E000E6B2101C0E9FF8F
:102D1000EA6EEFCF70F70C0E6A25016E000E6B2184
:102D200001C0E9FFEA6E6CC7EFFF716B7051715D16
:102D3000D8B07ED06AC7E9FF6BC7EAFFEFCF00F0DB
:102D4000ECCF01F0ECCF02F0ECCF03F06FC7EAFF5D
:102D50006EC7E9FF00C0EFFF01C0ECFF02C0ECFF4F
:102D600003C0ECFF6BC79AF76AC799F7060E9B6F13
:102D7000000185EC09F001C06DF707016D2D01D050
:102D800012D0726B7251000144EC03F00701722BF8
:102D9000006E00509EA8FED7AD6E340E725DF2E15B
:102DA000FF0E016E79D00601FB531AE107016AC7D5
:102DB000E9FF6BC7EAFFEFCF00F0020EEC24016ED3
:102DC000000EEC20026E000EEC20ED52ED52ED52A2
:102DD00000C0EFFF01C0ECFF02C0ECFFEC6E15D0AD
:102DE00007016AC701F06BC703F06AC772F76BC7C8
:102DF00073F76AC7E9FF6BC7EAFF010EEE2605E12C
:102E0000EE2A03E1EE2A01E1ED2A020E7125006EA1
:102E1000D89000360050036A290FE96E060E032091
:102E2000EA6EF0C6ECFFED52EFC6EFFF712B7ED7D6
:102E30006BC79AF76AC799F7070E9B6F000185EC7D
:102E400009F001C06DF7020E07017025006ED890E1
:102E500000360050036A290FE96E060E0320EA6E61
:102E6000F0C6ECFFED52EFC6EFFF6D51030812E123
:102E7000726B7251000103EC02F00701722B006EBD
:102E800000509EA8FED7AD6E110E725DF2E1FF0EEE
:102E9000016E02D0010E016E000170EF28F00701F3
:102EA0006B536BE1126B116B106B0F6B146B230E7A
:102EB000136F186B010E176F1B6F070E9A6F0F0EB3
:102EC000996F010E9B6F000185EC09F001C06CF752
:102ED000E5C1EBF607016F6B030E6E6F6F510308D0
:102EE0001BE372C773F771C772F770C771F7706B26
:102EF000C60E6E25746F010E756FD8B0752B230E3C
:102F00007425E96E000E7521EA6EEFCF6DF76D51F5
:102F100070136E076F2BE2D773C780F672C77FF608
:102F200071C77EF670C77DF66F6B030E6E6F6F51C3
:102F300003081BE372C773F771C772F770C771F7A5
:102F4000706BCA0E6E25746F010E756FD8B0752B3D
:102F5000230E7425E96E000E7521EA6EEFCF6DF732
:102F60006D5170136E076F2BE2D773C77CF672C773
:102F70007BF671C77AF670C779F66B2D2ED080C6B6
:102F800012F77FC611F77EC610F77DC60FF7060150
:102F9000FB530CE1D89011C712F710C711F70FC7F8
:102FA00010F707010F6B1037113712370701146B39
:102FB000230E136F186B010E176F1B6F070E9A6F9E
:102FC0000F0E996F010E9B6F000185EC09F001C097
:102FD0006CF707016CC701F002D0000E016E000112
:102FE000000C0701736B320E726F716B706B6F6B3D
:102FF0006E6B73C703F07251D8B473077207E96E32
:1030000003C0EAFFEFCF6CF7776B77C770F76CC739
:103010006FF76E6B716B72C7E9FF73C7EAFFEF5012
:103020006E136E5106017D25816F07016F510601F8
:103030007E21826F0701705106017F21836F070196
:10304000715106018021846F0701736B370E726F17
:103050006D6B716B706B6F6B6E6B6D51030816E36C
:1030600070C771F76FC770F76EC76FF76E6B73C776
:1030700003F07251D8B473077207E96E03C0EAFF18
:10308000EFCF6CF76C516E136D2BE7D771C78CF6D1
:1030900070C78BF66FC78AF66EC789F6060E756F16
:1030A0008D0E746F080E7425E96E000E7521EA6EA0
:1030B000EF6A0601895306E18A5304E18B5302E16A
:1030C0008C5344E00701736B3A0E726F6D6B716B3A
:1030D000706B6F6B6E6B6D51010816E370C771F703
:1030E0006FC770F76EC76FF76E6B73C703F07251DF
:1030F000D8B473077207E96E03C0EAFFEFCF6CF72D
:103100006C516E136D2BE7D7736B590E726F6D6B2D
:103110006D51070819E3036A6D517425016E7551ED
:10312000032203C077F7036A6D517225E96E73516C
:103130000320EA6EEFCF78F777C7EAFF01C0E9FF17
:1031400078C7EFFF6D2BE4D743D006010701736BFF
:103150004A0E726F6D6B716B706B6F6B6E6B6D5136
:10316000030816E370C771F76FC770F76EC76FF784
:103170006E6B73C703F07251D8B473077207E96EB0
:1031800003C0EAFFEFCF6CF76C516E136D2BE7D7DE
:10319000736B750E726F6D6B6D51070819E3036ADF
:1031A0006D517425016E7551032203C077F7036AD0
:1031B0006D517225E96E73510320EA6EEFCF78F7F7
:1031C00077C7EAFF01C0E9FF78C7EFFF6D2BE4D7AF
:1031D0006E5106018125856F07016F51060182211D
:1031E000866F0701705106018321876F07017151B6
:1031F00006018421886F07016E51060185259D6FA8
:1032000007016F51060186219E6F0701705106016B
:1032100087219F6F0701715106018821A06F71C737
:103220009CF670C79BF66FC79AF66EC799F6A46BAB
:10323000A36BA26B30C0A1F6A86BA76BA66B4FC0A7
:10324000A5F6030EEC6FC56BA0C6C0F69FC6BFF611
:103250009EC6BEF69DC6BDF6895306E18A5304E1BB
:103260008B5302E18C5306E0C46BC36BC26B020E3E
:10327000C16F05D0C46BC36BC26B4FC0C1F689531D
:1032800006E18A5304E18B5302E18C5315E0200ED2
:103290009D2507016E6F000E06019E2107016F6FCD
:1032A000000E06019F210701706F000E0601A0218C
:1032B0000701716F14D00601A1519D2507016E6FA2
:1032C0000601A2519E2107016F6F0601A3519F21A4
:1032D0000701706F0601A451A0210701716F71C72A
:1032E000BCF670C7BBF66FC7BAF66EC7B9F671C742
:1032F00003F770C702F76FC701F76EC700F7010E3B
:10330000016E00012EEF1AF007016B6B0001C7DDA3
:1033100001C06AF707016A51FF08D8B489D06B6B06
:103320006B510001A5EC03F007016B2B006E005000
:103330009EA8FED7AD6E100E6B5DF2E180C6ADF7B4
:10334000370EAE6F000176EC05F07FC6ADF7370E95
:103350000701AE6F000176EC05F07EC6ADF7370EC3
:103360000701AE6F000176EC05F07DC6ADF7370EB4
:103370000701AE6F000176EC05F0130E07016C6FCC
:103380006C510001A5EC03F007016C2B006E00509E
:103390009EA8FED7AD6E260E6C5DF2E17CC6ADF741
:1033A000370EAE6F000176EC05F07BC6ADF7370E39
:1033B0000701AE6F000176EC05F07AC6ADF7370E67
:1033C0000701AE6F000176EC05F079C6ADF7370E58
:1033D0000701AE6F000176EC05F00D0E9EA8FED73A
:1033E000AD6E0A0E9EA8FED7AD6EEBC66BF7070159
:1033F0006C6B6C510001C8EC03F007016C2B006E84
:1034000000509EA8FED7AD6E160E6C5DF2E16BC744
:10341000ADF7370EAE6F000176EC05F00D0E9EA8ED
:10342000FED7AD6E0A0E9EA8FED7AD6E04D0070182
:10343000000E016E4DD1010E07016B6F00012FDDF3
:1034400001C06AF707016A51FF08D8B43FD1030EE3
:103450000601EC6F07016B6B0001C3D501C06AF771
:1034600007016A2D33D16B6B6B510001E3EC03F064
:1034700007016B2B006E00509EA8FED7AD6E0F0E9D
:103480006B5DF2E184C6ADF7370EAE6F000176ECEE
:1034900005F083C6ADF7370E0701AE6F000176EC7D
:1034A00005F082C6ADF7370E0701AE6F000176EC6E
:1034B00005F081C6ADF7370E0701AE6F000176EC5F
:1034C00005F0120E07016C6F6C510001E3EC03F084
:1034D00007016C2B006E00509EA8FED7AD6E210E2A
:1034E0006C5DF2E19CC6ADF7370EAE6F000176EC75
:1034F00005F09BC6ADF7370E0701AE6F000176EC05
:1035000005F09AC6ADF7370E0701AE6F000176ECF5
:1035100005F099C6ADF7370E0701AE6F000176ECE6
:1035200005F0240E07016D6F6D510001E3EC03F00F
:1035300007016D2B006E00509EA8FED7AD6E2E0EBB
:103540006D5DF2E16B6B6B51000108EC04F007015B
:103550006B2B006E00509EA8FED7AD6E0F0E6B5DFC
:10356000F2E1A0C6ADF7370EAE6F000176EC05F0C4
:103570009FC6ADF7370E0701AE6F000176EC05F080
:103580009EC6ADF7370E0701AE6F000176EC05F071
:103590009DC6ADF7370E0701AE6F000176EC05F062
:1035A000120E07016C6F6C51000108EC04F007016A
:1035B0006C2B006E00509EA8FED7AD6E2C0E6C5D7D
:1035C000F2E1A4C6ADF7370EAE6F000176EC05F060
:1035D000A3C6ADF7370E0701AE6F000176EC05F01C
:1035E000A2C6ADF7370E0701AE6F000176EC05F00D
:1035F000A1C6ADF7370E0701AE6F000176EC05F0FE
:103600000D0E9EA8FED7AD6E0A0E9EA8FED7AD6E1B
:1036100007016B6B6B5100012EEC04F007016B2B63
:10362000006E00509EA8FED7AD6E0F0E6B5DF2E1EE
:10363000BCC6ADF7370EAE6F000176EC05F0BBC629
:10364000ADF7370E0701AE6F000176EC05F0BAC694
:10365000ADF7370E0701AE6F000176EC05F0B9C685
:10366000ADF7370E0701AE6F000176EC05F02C0EBA
:103670009EA8FED7AD6E200E9EA8FED7AD6E0701A8
:103680006B6B6B51000146EC04F007016B2B006E75
:1036900000509EA8FED7AD6E0D0E6B5DF2E1060EDA
:1036A000EA6E8D0EE96E000EEF1008E0EF509EA856
:1036B000FED7AD6EE92AD8B4EA2AF5D70D0E9EA83A
:1036C000FED7AD6E0A0E9EA8FED7AD6E000E016E3F
:1036D00000018CEF28F007016A6B6A5100014FEC82
:1036E00000F007016A2B006E00509EA8FED7AD6E59
:1036F0002B0E6A5DF2E10001000C07016A6B6A5152
:10370000000172EC00F007016A2B006E00509EA8C9
:10371000FED7AD6E340E6A5DF2E10001000C0701C8
:10372000906B8F6B8E6B8D6B8BC703F08A518A2BDE
:10373000D8B48B2BE96E03C0EAFFEFCF8CF78CC7B0
:1037400092F70001E5EC13F001C091F70701913DFC
:103750000FD088C7E9FF89C7EAFF8DC7EFFF8EC783
:10376000ECFF8FC7ECFF90C7ECFF8CC701F017D0C0
:103770008D378E378F3790378D378E378F3790371D
:103780008D378E378F3790378D378E378F3790370D
:10379000F00E8D1791518D13C7D7000E016E0001E9
:1037A000EBEF1CF00701876B6CA504D0010E876F4F
:1037B000030E6C176C2D0CD06AC7E9FF6BC7EAFFCC
:1037C000ECCF03F0ED52EFCF6FF703C070F70BD0E3
:1037D0006AC7E9FF6BC7EAFFECCF03F0ED52EFCF0A
:1037E0006DF703C06EF70D0E9EA8FED7AD6E0A0EE4
:1037F0009EA8FED7AD6E6C2D11D070C7ADF7370EF9
:10380000AE6F000176EC05F06FC7ADF7370E07011C
:10381000AE6F000176EC05F010D007016EC7ADF772
:10382000370EAE6F000176EC05F06DC7ADF7370EC1
:103830000701AE6F000176EC05F03D0E9EA8FED7A5
:10384000AD6E070187532EE16C2D1CD070C703F0BD
:103850006FC7E9FF70C7EAFFECCF89F7ED52EFCFF2
:1038600088F789C7ADF7370EAE6F000176EC05F02B
:1038700088C7ADF7370E0701AE6F000176EC05F093
:1038800010D007016EC703F06DC7E9FF6EC7EAFFEE
:10389000EFCF88F788C7ADF7370EAE6F000176EC33
:1038A00005F00701200E9EA8FED7AD6E070E896FAA
:1038B000710E886F0F0E8A6F010E8B6F000117EC6F
:1038C0000FF00701826B01C081F7813D05D0825363
:1038D00003E1000E016EA7D0825303E181510F086E
:1038E00062E28151520802E1825305E0815172087F
:1038F0000EE182530CE16C2D05D0FE0E6F27D8A08F
:10390000700704D06D51D8B46E076D0749D081514E
:10391000580802E1825305E08151780837E182536B
:1039200035E1872D33D06C2D1CD070C703F06FC7E5
:10393000E9FF70C7EAFFECCF89F7ED52EFCF88F7C8
:1039400089C7ADF7370EAE6F000176EC05F088C77A
:10395000ADF7370E0701AE6F000176EC05F010D021
:1039600007016EC703F06DC7E9FF6EC7EAFFEFCF2F
:1039700088F788C7ADF7370EAE6F000176EC05F01B
:10398000200E9EA8FED7AD6E0CD007016C2D05D081
:10399000020E6F27D8B0702B03D06D2BD8B46E2BCE
:1039A00000013DD00701070E866F710E856F86C737
:1039B00003F085C7E9FF86C7EAFFEF502E0801E153
:1039C00030D0070E896F830E886F86C78BF785C747
:1039D0008AF70001A4D684C782F783C781F707015D
:1039E0006C2D12D070C703F06FC700F0020E6F2766
:1039F000D8B0702B00C0E9FF03C0EAFF82C7ECFF1C
:103A0000ED5281C7EFFF0BD06EC703F06D516D2BE8
:103A1000D8B46E2BE96E03C0EAFF81C7EFFF070140
:103A2000E2D6000E016E00010DEF2BF0EACF90F709
:103A3000E9CF8FF707018939F0098B6F8B27E20FE8
:103A40008C6F320F8E6F89510F0B8C278C278E272E
:103A5000E90F8D6F8D278D2788390F0B8D278E27C6
:103A60008D378E378E1F8E3788510F0B8E278B37F1
:103A7000070E8A6F0A0E8D078E27FDE38C078D27B0
:103A8000FDE38B078C27FDE38A078B27FDE3070EF9
:103A9000EA6E8A0EE96E070E8F158F9DE9268E0E4F
:103AA000E95CD8B48F8DEF50006E08E18FBD06D071
:103AB0008FB916D08FB702D0200E03D08F878F9981
:103AC000300E0026EACF89F7E9CF88F700C0ADF7BE
:103AD00000012BEC08F089C7EAFF88C7E9FF07015E
:103AE000EE508FADDCD70001DDEF1FF007016AC794
:103AF000E9FF6BC7EAFFEFCF6CF7020E756F230E7D
:103B0000746F706B84C687F783C686F782C685F7A5
:103B100081C684F788C683F787C682F786C681F791
:103B200085C680F7040E6A25016E000E6B2101C068
:103B3000E9FFEA6E020EEC6EED52230EEF6E080EF8
:103B40006A25016E000E6B2101C0E9FFEA6E010ECD
:103B5000EF6E0C0E6A25016E000E6B2101C0E9FFAD
:103B6000EA6E010EEF6E6E6B796B786B776B766F2A
:103B70006E516C5DD8A029D16D6B6D510708D8A02E
:103B80001FD16C516E5D6EE16D536CE174C7E9FF3E
:103B900075C7EAFF79C703F078C702F077C701F06D
:103BA00076C700F0010E7627D8B0772BD8B4782BE3
:103BB000D8B4792B00C0EFFF01C0ECFF02C0ECFFCE
:103BC00003C0ECFF040E7425E96E000E7521EA6E49
:103BD00079C703F078C702F077C701F076C700F025
:103BE000010E7627D8B0772BD8B4782BD8B4792BA0
:103BF00000C0EFFF01C0ECFF02C0ECFF03C0ECFF10
:103C0000080E7425E96E000E7521EA6EFF0EEF6E48
:103C1000EC6EEC6E0F0EEC6E7F6B030E7E6F7F53BF
:103C20001EE17E517F081BE37E35026E7F35036EF9
:103C300002360336FC0E021602507425E96E7551E9
:103C40000320EA6EEE52EE52EC6AED52EF6AED524C
:103C5000EF6AED52EF6A7E2BD8B47F2BE0D7010ECE
:103C6000706F64D07F6B7E6B7F532DE17E517F0838
:103C70002AE37E35026E7F35036E02360336FC0E74
:103C8000021602507425E96E75510320EA6E79C759
:103C900003F078C702F077C701F076C700F0010E95
:103CA0007627D8B0772BD8B4782BD8B4792B00C02E
:103CB000EFFF01C0ECFF02C0ECFF03C0ECFF7E2B66
:103CC000D8B47F2BD1D76D5331E16E5323E174C744
:103CD000E9FF75C7EAFFF80EEF6EFF0EEC6EEC6EB3
:103CE0000F0EEC6E040E7425E96E000E7521EA6E5F
:103CF000FF0EEF6EEC6EEC6EEC6E080E7425E96E46
:103D0000000E7521EA6EFF0EEF6EEC6EEC6E0F0E7C
:103D1000EC6E0CD0080E7425E96E000E7521EA6E6B
:103D2000FF0EEF6EEC6EEC6E0F0EEC6E6AC7E9FFE5
:103D30006BC7EAFF84C7EFFF85C7ECFF86C7ECFFC0
:103D400087C7ECFF6BC79AF76AC799F7020E9B6F9C
:103D5000000185EC09F001C06FF707016F2D01D05C
:103D600003D06FC701F06DD26AC7E9FF6BC7EAFFE6
:103D700080C7EFFF81C7ECFF82C7ECFF83C7ECFF72
:103D80006BC79AF76AC799F7020E9B6F000185EC23
:103D900009F001C06FF707016F2D01D003D06FC785
:103DA00001F04FD2010E8427000E8523862387233E
:103DB000010E8027000E8123822383236D2BDDD605
:103DC000705301E002D06E2BD3D6060199518125A4
:103DD0000701766F06019A5182210701776F06016C
:103DE0009B5183210701786F06019C5184210701B3
:103DF000796F7F6B7E6B7F51010818E3040E6A2593
:103E0000016E000E6B2101C0E9FFEA6EECCF8DF769
:103E1000ED52EFCF8CF78C517E25E96E8D517F21CD
:103E2000EA6EEF6A7E2BD8B47F2BE5D78751795D98
:103E300057E30BE18651785D53E307E18551775DE8
:103E40004FE303E17651845D4BE26AC7E9FF6BC73C
:103E5000EAFF84C7EFFF85C7ECFF86C7ECFF87C783
:103E6000ECFF6BC79AF76AC799F7020E9B6F0001C8
:103E700085EC09F001C06FF707016F2D01D003D069
:103E80006FC701F0DED16AC7E9FF6BC7EAFF80C7E1
:103E9000EFFF81C7ECFF82C7ECFF83C7ECFF6BC766
:103EA0009AF76AC799F7020E9B6F000185EC09F03B
:103EB00001C06FF707016F2D01D003D06FC701F06C
:103EC000C0D1010E8027000E812382238323010E9F
:103ED0008427D8B0852BD8B4862BD8B4872BA6D707
:103EE00000012DEC07F003C07DF702C07CF701C094
:103EF0007BF700C07AF70701886B8851000185ECD9
:103F000004F00701882B006E00509EA8FED7AD6E0E
:103F1000090E885DF2E17DC7ADF7370EAE6F000187
:103F200076EC05F07CC7ADF7370E0701AE6F0001E8
:103F300076EC05F07BC7ADF7370E0701AE6F0001D9
:103F400076EC05F07AC7ADF7370E0701AE6F0001CA
:103F500076EC05F0A0C687F79FC686F79EC685F764
:103F60009DC684F70701796B786B776B030E766FCC
:103F70006C3B0F0E6C177F6B7E6B010E716F6E6B5F
:103F80006C516E5DD8B0FDD0020E736F230E726F50
:103F90006D6B6D510F08D8A0CBD073C758F772C79F
:103FA00057F7440EAD6F00012BEC08F0090EE96ED7
:103FB0007FC789F77EC788F739D5060E0701886F56
:103FC0008851000199EC04F00701882B006EAD6F59
:103FD00000012BEC08F00D0E0701885DF1E17E2B4E
:103FE000D8B47F2B715379E00C0E7225E96E000E68
:103FF0007321EA6EEF6A0D0E7225E96E000E7321D1
:10400000EA6EEF6A0E0E7225E96E000E7321EA6EFB
:104010007AC7EFFF0F0E7225E96E000E7321EA6E6C
:104020007BC7EFFF100E7225E96E000E7321EA6E5A
:104030007CC7EFFF110E7225E96E000E7321EA6E48
:104040007DC7EFFF120E7225E96E000E7321EA6E36
:10405000EF6A130E7225E96E000E7321EA6EEF6AA5
:10406000160E7225E96E000E7321EA6E7AC7EFFF15
:10407000170E7225E96E000E7321EA6E7BC7EFFF03
:10408000180E7225E96E000E7321EA6E7CC7EFFFF1
:10409000190E7225E96E000E7321EA6E7DC7EFFFDF
:1040A0001C0E7225E96E000E7321EA6EEF6A1D0E7A
:1040B0007225E96E000E7321EA6EEF6A1E0E7225FC
:1040C000E96E000E7321EA6EEF6A1F0E7225E96E2B
:1040D000000E7321EA6E020EEF6E140E7225E96E69
:1040E000000E7321EA6E78C7EFFF150E7225E96E98
:1040F000000E7321EA6E79C7EFFF1A0E7225E96E82
:10410000000E7321EA6E76C7EFFF1B0E7225E96E73
:10411000000E7321EA6E77C7EFFF040E7727000EBB
:1041200078237923200E7227000E73236D2B31D74D
:10413000716B6AC7E9FF6BC7EAFF84C7EFFF85C7EA
:10414000ECFF86C7ECFF87C7ECFF6BC79AF76AC71F
:1041500099F7020E9B6F000185EC09F001C06FF723
:1041600007016F2D01D003D06FC701F06AD0010E97
:104170008427D8B0852BD8B4862BD8B4872B6E2B48
:10418000FFD6020E736F230E726F7F6B7E6B7F51B3
:1041900001080BE372517E25E96E73517F21EA6EAF
:1041A000EF6A7E2BD8B47F2BF2D70601A1519D2553
:1041B0000701766F0601A2519E210701776F060164
:1041C000A3519F210701786F0601A451A021070187
:1041D000796F8751795D33E30BE18651785D2FE389
:1041E00007E18551775D2BE303E17651845D27E29A
:1041F0006AC7E9FF6BC7EAFF84C7EFFF85C7ECFF1B
:1042000086C7ECFF87C7ECFF6BC79AF76AC799F7B9
:10421000020E9B6F000185EC09F001C06FF70701EA
:104220006F2D01D003D06FC701F00BD0010E842792
:10423000D8B0852BD8B4862BD8B4872BCAD7010E1B
:10424000016E000189EF2AF0F86AD09E0D8EEA6AAD
:10425000E96AB886220EAF6E000EB06EA60EAC6E86
:10426000900EAB6EC150C00B0F09C16E070EB46E3D
:10427000030E186E196A1A6A0701576B586BAB8EDA
:10428000AB889380FF0E946E82909392819281947A
:104290009384080E6F6E070E1C6EDC0E1B6E040EF0
:1042A0001D6E070E1E6E130E1F6E1E0E206E216AEF
:1042B0000601EC6BC50ED56E830EFA6FD76AD66A0F
:1042C000F28AC00EF212C150C00B0D09C16EC0803F
:1042D000C082C084C08EC280000E016EC250C30B6B
:1042E0000110C26EFD6B020EFF6F0C0EFE6FF06BC5
:1042F000EF6B0701046B0B6B6A6B6A51000123ECD7
:1043000001F007016A2B006E00509EA8FED7AD6E2B
:104310002C0E6A5DF2E1AD6B370EAE6F000176ECEC
:1043200005F0230E0701AD6F370EAE6F000176EC7E
:1043300005F02FEC06F0D5EC06F007016A6B6A5128
:10434000000148EC01F007016A2B006E00509EA8A6
:10435000FED7AD6E0D0E6A5DF2E1070E896F2F0E6E
:10436000886F270E8A6F8B6B000117EC0FF001C06E
:1043700059F707015951FF0801E1E0D7070E626FB5
:104380002F0E616F61C7E9FF62C7EAFFEFCF63F7E6
:1043900063511B0A00012DE0220A58E00A0AD8B432
:1043A000AAD0520AD8B443D1040AD8B46ED11D0A97
:1043B000D8B489D1110AD8B4CCD1050AD8B4F9D16E
:1043C0003F0AD8B4F8D2370AD8B4BAEF28F0170A9F
:1043D000D8B474EF29F0350AD8B4A1EF29F02E0A29
:1043E000D8B4A3EF2AF0110AD8B4D6EF2AF00DEF13
:1043F0002BF0010E07010A5DFB0F24E2050F0001FF
:1044000012EF2BF007010B2B0B51010801E20B6B94
:10441000010E6A6F000140EC13F0070113D0020E89
:1044200007016A6F000140EC13F007010BD0030E87
:1044300007016A6F000140EC13F0070103D0070188
:1044400001D007010A6B00010DEF2BF0490E0701A7
:10445000AB6FAF6BAE6BAD6BAC6B00014EEC09F0AC
:1044600007015B6B5B5109080EE3FF0EB56F00019E
:1044700030EC09F001C05AF707015A51800B01E1F5
:1044800002D05B2BEFD76A6B6A5100015CEC01F044
:1044900007016A2B006E00509EA8FED7AD6E0D0E70
:1044A0006A5DF2E15AC7ADF7370EAE6F000176ECE8
:1044B00005F0200E9EA8FED7AD6E0701596B59512D
:1044C000190816E3FF0EB56F000130EC09F001C0CA
:1044D0005AF75AC7ADF7370E0701AE6F000176ECF9
:1044E00005F0200E9EA8FED7AD6E0701592BE7D729
:1044F00000010DEF2BF0770E0701AB6FAF6BAE6BCA
:10450000AD6BAC6B00014EEC09F00701596B5951D2
:1045100009080EE3FF0EB56F000130EC09F001C091
:104520005AF707015A51800B01E102D0592BEFD7FE
:104530006A6B6A51000172EC01F007016A2B006E90
:1045400000509EA8FED7AD6E0E0E6A5DF2E15AC70E
:10455000ADF7370EAE6F000176EC05F0200E9EA889
:10456000FED7AD6E4D0E0701AB6FAF6BAE6BAD6B93
:10457000AC6B00014EEC09F00701596B5951090869
:104580000EE3FF0EB56F000130EC09F001C05AF7E1
:1045900007015A51800B01E102D0592BEFD76A6B0A
:1045A0006A51000188EC01F007016A2B006E00508F
:1045B0009EA8FED7AD6E0F0E6A5DF2E15AC7ADF749
:1045C000370EAE6F000176EC05F0200E9EA8FED7E8
:1045D000AD6E0D0E9EA8FED7AD6E0A0E9EA8FED73C
:1045E000AD6E0701596B595147081EE3FF0EB56FB9
:1045F000000130EC09F001C05AF75AC7ADF7370E89
:104600000701AE6F000176EC05F0200E9EA8FED7E4
:10461000AD6E070159510F0B0F0804E10001DCECEE
:1046200013F00701592BDFD700010DEF2BF0070125
:10463000612BD8B4622B62C76BF761C76AF7070EAC
:104640006D6F0F0E6C6F010E6E6F6F6B000102ECE1
:1046500014F001C059F707010F35006E0036FC0E4B
:104660000016C250C30B0010C26EC282C2B2FED787
:10467000C3CF5FF7C4CF60F760C76BF75FC76AF758
:10468000000134EC15F00DEF2BF0D6500701596FF7
:10469000C282C2B2FED7C3CF5FF7C4CF60F760C794
:1046A0009CF75FC79BF70001C8EC08F0D6500701E4
:1046B0006A6F59516A5D596F59C76AF70001AEECCC
:1046C00015F00DEF2BF00701612BD8B4622B62C7F8
:1046D0006BF761C76AF7070E6D6F0F0E6C6F010EF7
:1046E0006E6F6F6B000102EC14F001C059F712C736
:1046F0009CF711C79BF710C79AF70FC799F713C715
:104700009DF731EC0DF018C79CF717C79BF7C8EC65
:1047100008F0070E0701586F460E576F6A6B6A5113
:104720000001A0EC01F007016A2B006EAD6F0001E3
:104730002BEC08F0070E07016A5DF1E1490E806F6E
:10474000070E826F460E816F0001A3EC0FF00DEF94
:104750002BF00701612BD8B4622B5A6B62C703F0B0
:1047600061C7E9FF62C7EAFFEF50690805E1612B05
:10477000D8B4622B010E5A6F62C76BF761C76AF734
:10478000070E6D6F0F0E6C6F010E6E6F6F6B000179
:1047900002EC14F001C059F707015A2D05D00001B1
:1047A0002FEC06F004D007010001D5EC06F00DEF68
:1047B0002BF00701612BD8B4622B62C703F061C7ED
:1047C000E9FF62C7EAFFEF50730868E16A6B6A515C
:1047D0000001B1EC01F007016A2B006E00509EA8A9
:1047E000FED7AD6E0D0E6A5DF2E104C76CF71F0EC9
:1047F0006D6F000140EC15F00F0E07016B6F6B51F0
:104800000001B1EC01F007016B2B006E00509EA877
:10481000FED7AD6E1B0E6B5DF2E1FFC6ADF7370E36
:10482000AE6F000176EC05F0FEC6ADF7370E07015E
:10483000AE6F000176EC05F007016A6B6A5100016A
:10484000CEEC01F007016A2B006E00509EA8FED747
:10485000AD6E130E6A5DF2E103C7ADF7370EAE6FB2
:10486000000176EC05F002C7ADF7370E0701AE6F19
:10487000000176EC05F001C7ADF7370E0701AE6F0A
:10488000000176EC05F000C7ADF7370E0701AE6FFB
:10489000000176EC05F00DEF2BF0070162C76BF716
:1048A00061C76AF7070E6D6F0F0E6C6F010E6E6FAA
:1048B0006F6B000102EC14F001C059F707010FA360
:1048C00034D00601EC51030B030813E007016A6BB7
:1048D0006A510001E7EC01F007016A2B006E0050FD
:1048E0009EA8FED7AD6E1C0E6A5DF2E100010DEFD1
:1048F0002BF00701045318E1006A016A0050060119
:10490000B9250701006F01500601BA210701016FA7
:1049100013510601BB210701026F14510601BC218E
:104920000701036F010E046F41D0045102081FE11B
:10493000070E9A6F1F0E996F070E9B6F000185EC93
:1049400009F001C059F707015951030810E16A6BDA
:104950006A51000103EC02F007016A2B006E00505F
:104960009EA8FED7AD6E110E6A5DF2E1046B046B7A
:10497000070E586F460E576F6A6B6A510001A0EC24
:1049800001F007016A2B006EAD6F00012BEC08F0FF
:10499000070E07016A5DF1E1490E806F070E826F15
:1049A000460E816F0001A3EC0FF007010FC7FDF663
:1049B00000010DEF2BF00701612BD8B4622B62C709
:1049C00003F061C7E9FF62C7EAFFEF506908D8A4A6
:1049D00083D25A6B5A51090808E3FF0EB56F0001E4
:1049E00030EC09F007015A2BF5D7400EAB6FAF6BD7
:1049F000AE6BAD6BAC6B00014EEC09F007015B6B6D
:104A00005B5109080EE3FF0EB56F000130EC09F0B1
:104A100001C05AF707015A51800B01E102D05B2B0C
:104A2000EFD76A6B6A51000119EC02F007016A2B9B
:104A3000006E00509EA8FED7AD6E080E6A5DF2E1D2
:104A40005AC76BF70001BAEC15F0010E0701B06F01
:104A5000000128EC09F0FF0E0701B56F000130ECF2
:104A600009F007015E6B0A0E5D6F5EC703F05D51D2
:104A7000D8B45E075D0703103BE0480E6A6F6E6BAB
:104A80006D6B010E6C6FAA0E6B6F870E6F6F00015E
:104A9000C3EF15F007015B6B5B5109080EE3FF0ED6
:104AA000B56F000130EC09F001C05AF707015A5107
:104AB000800B01E102D05B2BEFD75B6B5B510508EC
:104AC00008E3FF0EB56F000130EC09F007015B2B26
:104AD000F5D75A2D01D002D05AA501D009D09EAAEF
:104AE00006D09EAAFED7AE50030801E101D0BDD783
:104AF0006A6B6A5100012BEC02F007016A2B006E11
:104B000000509EA8FED7AD6E080E6A5DF2E15AC74E
:104B10006BF70001BAEC15F0010E0701B06F000150
:104B200028EC09F0FF0E0701B56F000130EC09F029
:104B300007015E6B5D6B7A0EAB6FAF6BAE6BAD6BEF
:104B4000AC6B00014EEC09F007015B6B5B5109088F
:104B50000EE3FF0EB56F000130EC09F001C05AF70B
:104B600007015A51800B01E102D05B2BEFD75B6B41
:104B70005B51050818E3036A5B51230F016E060EB3
:104B8000032201C06AF703C06BF7FF0EB56F000187
:104B900030EC09F06BC7EAFF6AC7E9FF01C0EFFF1D
:104BA00007015B2BE5D79EAA0CD09EAAFED7AE507C
:104BB000030807E15AC76BF70001BAEC15F016D0ED
:104BC00007015D2BD8B45E2B010EB06F000128ECFD
:104BD00009F0FF0E0701B56F000130EC09F0070185
:104BE0005A2D03D0000102D00701A5D707016A6B37
:104BF0006A5100013DEC02F007016A2B006E005083
:104C00009EA8FED7AD6E090E6A5DF2E15B6B5B514B
:104C1000030811E3036A5B51230FE96E060E0320BC
:104C2000EA6EEFCF6AF76AC76BF70001BAEC15F0CE
:104C300007015B2BECD75E6B5D6B770EAB6FAF6BD9
:104C4000AE6BAD6BAC6B00014EEC09F007015B6B1A
:104C50005B5109080DE3FF0EB56F000130EC09F060
:104C600001C05AF707015A2D01D002D05B2BF0D7B3
:104C7000FF0EB56F000130EC09F0690E0701AB6F54
:104C8000400EAF6FFF0EAE6F800EAD6FAC6B0001CC
:104C90004EEC09F007015B6B5B51090810E3FF0E56
:104CA000B56F000130EC09F001C05AF707015A5303
:104CB00001E105D05A2D01D002D05B2BEDD75AC7A8
:104CC00023F6010E5B6F5B51050818E3036A5B5125
:104CD000230F016E060E032201C06AF703C06BF7B3
:104CE000FF0EB56F000130EC09F06BC7EAFF6AC731
:104CF000E9FF01C0EFFF07015B2BE5D79EAA1BD0A0
:104D00009EAAFED7AE50030816E15B6B5B51050807
:104D100011E3036A5B51230FE96E060E0320EA6E6E
:104D2000EFCF6AF76AC76BF70001BAEC15F007011D
:104D30005B2BECD71FD05D2BD8B45E2B010EB06F70
:104D4000000128EC09F0FF0E0701B56F000130ECFF
:104D500009F007015A5307E1060124BF02D00701F9
:104D600002D0070107D0640E6C6F000199EC05F0CA
:104D7000070163D76A6B6A5100014FEC02F007012B
:104D80006A2B006E00509EA8FED7AD6E0A0E6A5DBB
:104D9000F2E16B6B5AC76AF75DC703F0000E5A2544
:104DA0006C6F5D516B216D6F6F6F6CC76EF700019B
:104DB00001EF16F07A0E0701AB6FAF6BAE6BAD6B08
:104DC000AC6B00014EEC09F007015B6B5B5109080D
:104DD0000DE3FF0EB56F000130EC09F001C05AF78A
:104DE00007015A5301E102D05B2BF0D75B6B5B519B
:104DF000050818E3036A5B51230F016E060E0322B8
:104E000001C06AF703C06BF7FF0EB56F000130EC0D
:104E100009F06BC7EAFF6AC7E9FF01C0EFFF0701AE
:104E20005B2BE5D79EAA06D09EAAFED7AE500308FC
:104E300001E119D05D2BD8B45E2B010EB06F0001DB
:104E400028EC09F0FF0E0701B56F000130EC09F006
:104E500007015A5305E1010E0601EC6F070103D06B
:104E60000001A8D707016A6B6A5100013DEC02F00E
:104E700007016A2B006E00509EA8FED7AD6E090E8A
:104E80006A5DF2E1060123AD03D0010EFB6F01D094
:104E9000FB6B07015B6B5B51030811E3036A5B511A
:104EA000230FE96E060E0320EA6EEFCF6AF76AC79A
:104EB0006BF70001BAEC15F007015B2BECD7010E84
:104EC000B06F000128EC09F0FF0E0701B56F00017B
:104ED00030EC09F04CD1070162C703F061C7E9FF6C
:104EE00062C7EAFFEF50720852E1612BD8B4622B1F
:104EF0005C6B62C703F061C7E9FF62C7EAFFEF506E
:104F00006D0805E1010E5C6F612BD8B4622B62C79E
:104F10006BF761C76AF7070E6D6F0F0E6C6F010EAE
:104F20006E6F6F6B000102EC14F001C059F70701BE
:104F3000595305E1000113EC16F00DEF2BF00601BB
:104F4000FB530DE1D89011C712F710C711F70FC727
:104F500010F707010F6B10371137123706015CC7C6
:104F60001BF7FC6B070E07019A6F0F0E996F010E6E
:104F70009B6F000185EC09F00601FC5306E0FCC6BE
:104F80006AF7000125EC16F00601F2D0070162C7AE
:104F900003F061C7E9FF62C7EAFFEF50770847E116
:104FA000612BD8B4622B5C6B62C703F061C7E9FF69
:104FB00062C7EAFFEF506D0805E1010E5C6F612BDF
:104FC000D8B4622B62C76BF761C76AF7070E6D6FC3
:104FD0000F0E6C6F010E6E6F6F6B000102EC14F020
:104FE00001C059F70701595304E1000113EC16F011
:104FF00014D30601FB530DE1D89011C712F710C767
:1050000011F70FC710F707010F6B10371137123761
:1050100006015CC71BF7070E07019A6F0F0E996F09
:10502000020E9B6F000185EC09F0A1D0070162C759
:1050300003F061C7E9FF62C7EAFFEF5057085AE182
:10504000612BD8B4622B5C6B62C703F061C7E9FFC8
:1050500062C7EAFFEF506D0805E1010E5C6F612B3E
:10506000D8B4622B62C76BF761C76AF7070E6D6F22
:105070000F0E6C6F010E6E6F6F6B000102EC14F07F
:1050800001C059F70701595304E1000113EC16F070
:10509000C4D20601FB530CE1D89011C712F710C718
:1050A00011F70FC710F707010F6B103711371237C1
:1050B00007011A5307E1195305E1185303E117518A
:1050C000200805E21A6B196B186B200E176F070E7C
:1050D0006B6F0F0E6A6F5CC76CF7000141EF16F043
:1050E00001C059F7DCEC13F059C76BF7BAEC15F0B7
:1050F0003ED0070162C703F061C7E9FF62C7EAFF5C
:10510000EF506D080BE10601ECA103D0000184EF24
:1051100019F000016BEC1BF02AD0070162C703F005
:1051200061C7E9FF62C7EAFFEF50640821E10601A9
:10513000EC51030B03080BE0ECA104D000017DEC63
:105140001BF003D000016BEC1BF067D20601FC6B77
:1051500007016C6B6D6B6E6B000117EC10F00601B4
:10516000FC5306E0FCC66AF7000125EC16F00601C8
:10517000000153D20701612BD8B4622B5A6B62C76E
:1051800003F061C7E9FF62C7EAFFEF506D0805E170
:10519000010E5A6F612BD8B4622B62C76BF761C7DF
:1051A0006AF7070E6D6F0F0E6C6F010E6E6F6F6BEF
:1051B000000102EC14F001C059F707015A2D05D087
:1051C00010C765F70FC764F707D0656B230E646FD0
:1051D0000F516427105165235E6B5D6B5E51145D4A
:1051E000D8A080D004E113515D5DD8B07BD05D5173
:1051F0000F0B6A6F6B6B6A5324E16B5322E16451AE
:105200005D256A6F65515E216B6F0D0E9EA8FED7FE
:10521000AD6E0A0E9EA8FED7AD6E6BC7ADF7370E0A
:10522000AE6F000176EC05F06AC7ADF7370E0701E7
:10523000AE6F000176EC05F05EC760F75DC75FF703
:10524000070164515D25E96E65515E21EA6EEFCF7D
:105250006AF7200E9EA8FED7AD6E6AC7ADF7370E6F
:10526000AE6F000176EC05F007015D510F0B6A6F20
:105270006B6B6A510F0832E16B5330E1200E9EA830
:10528000FED7AD6E5B0E9EA8FED7AD6E5A6B5A511F
:105290000F0820E360C703F05F515F2BD8B4602B89
:1052A0006A6F64516A25E96E65510320EA6EEFCF9B
:1052B0005BF75B511F0808E25B517A0805E35B511D
:1052C0009EA8FED7AD6E04D02E0E9EA8FED7AD6E62
:1052D0005A2BDDD75D0E9EA8FED7AD6E5D2BD8B4E0
:1052E0005E2B7CD7000199D10701612BD8B4622BCA
:1052F0005A6B62C703F061C7E9FF62C7EAFFEF506C
:10530000770805E1010E5A6F612BD8B4622B62C792
:105310006BF761C76AF7070E6D6F0F0E6C6F010EAA
:105320006E6F6F6B000102EC14F001C059F7070EAD
:1053300007016B6F0F0E6A6F5AC76CF70001D2EF4F
:105340001BF00601EC51030B03080BE0EC51010BC1
:1053500003E100016BEC1BF000017DEC1BF05DD163
:105360000601A151400806E1A25304E1A35302E162
:10537000A45313E007016A6B6A51000162EC02F06A
:1053800007016A2B006E00509EA8FED7AD6E3B0E43
:105390006A5DF2E1000141D10601895306E18A53B9
:1053A00004E18B5302E18C5312E007016A6B6A51EE
:1053B00000018DEC02F007016A2B006E00509EA8E0
:1053C000FED7AD6E160E6A5DF2E1000126D107012F
:1053D000612BD8B4622B62C76BF761C76AF7070EFF
:1053E0006D6F0F0E6C6F010E6E6F6F6B000102EC34
:1053F00014F001C059F70601B951795D0701666FD4
:105400000601BA517A590701676F0601BB517B59F2
:105410000701686F0601BC517C590701696F68C7B5
:1054200000F069C701F0026A036A0350125D42E3AB
:105430000BE10250115D3EE307E10150105D3AE3DC
:1054400003E100500F5D36E368C76BF769C76CF77F
:105450006D6B6E6B6F6B6F510001A6EC02F0070174
:105460006F2B006E00509EA8FED7AD6E2B0E6F5DA9
:10547000F2E16EC7ADF7370EAE6F000176EC05F0C6
:105480006DC7ADF7370E0701AE6F000176EC05F082
:105490006CC7ADF7370E0701AE6F000176EC05F073
:1054A0006BC7ADF7370E0701AE6F000176EC05F064
:1054B000B4D007016A6B6A510001CBEC02F007011E
:1054C0006A2B006E00509EA8FED7AD6E360E6A5D48
:1054D000F2E16A6B6A510001F4EC02F007016A2BF9
:1054E000006E00509EA8FED7AD6E340E6A5DF2E1EC
:1054F0009EAAFED7AECF5AF75A51790803E00001B1
:105500008CD00701070E6B6F0F0E6A6F000176EFEC
:105510001DF001C059F707016A6B6A5100011CECCC
:1055200003F007016A2B006E00509EA8FED7AD6EF7
:10553000080E6A5DF2E159C7ADF7370EAE6F000194
:1055400076EC05F06AD00701612BD8B4622B62C7F4
:1055500003F061C7E9FF62C7EAFFEF5211E1000102
:10556000DCEC13F01FC06AF7AEEC15F020C06AF750
:10557000AEEC15F021C06AF7AEEC15F04ED0070185
:1055800062C76BF761C76AF7070E6D6F0F0E6C6F1E
:10559000030E6E6F010E6F6F000102EC14F00FC767
:1055A0001FF013C720F017C721F037D00701612B78
:1055B000D8B4622B62C703F061C7E9FF62C7EAFF94
:1055C000EF5213E10001DCEC13F01CC06BF71BC0C1
:1055D0006AF734EC15F01DC06AF7AEEC15F01EC08A
:1055E0006AF7AEEC15F019D0070162C76BF761C717
:1055F0006AF7070E6D6F0F0E6C6F030E6E6F010E64
:105600006F6F000102EC14F010C71CF00FC71BF005
:1056100013C71DF017C71EF000D0DCEC13F09DEF90
:1056200021F00300F2CF0EF0F29EE824F76AF7367D
:10563000490FF66E560EF7220A00F550FA6E080072
:10564000F5500EBEF28EF96E04441E4442442E44C0
:025650003E44D6
:020000040030CA
:0E00000000041E1E008381000FC00FE00F40A1
:00000001FF
